:02000000017B82
:20007B0075811E904D3F79007A007B437C0EEB4C601CE493A3CAC583CAC9C582C9F0A3CA1B
:20009B00C583CAC9C582C91BBBFFE31C80E0900E5AE4F0123FF212001B80FBC82581C82217
:2000BB00C92581C97A0022D083D082CF2581F581CFC082C08322CF2581F581CF22FBE0CBC9
:2000DB0022FCE0FBA3E0CC22FAE0F9A3E0CA2229F9E5F03AFA227C00CB30E7011CCB22752F
:2000FB00F00030E70215F022FDE493A3FEE493A3FF4E7009E493FE740193FF800BE493A39F
:20011B00B5050BE493B5F0068F838E82E473A380D8FEEBA4FD8EF0ECA4FCEB8EF0A4C5F013
:20013B002C2DC5F02231468EF0ED22C002C001AAF0F97E007D007F11C3E933F9EA33FADF01
:20015B0008F5F0E9D001D00222ED33FDEE33FEC3ED9BF5F0EE9C40E0ADF0FED380DBBB004F
:20017B000122C333C5F033C5F0DBF722BB000122C3C5F013C5F013DBF722240280022401C8
:20019B00C5F03400C5F022C394028003C39401C5F09400C5F02231A7F4C5F0F4C5F022459F
:2001BB00F07022042251094024801A5109401E7014801A5109400E7014800A5109500E8060
:2001DB0004511D6008E4F5F022511D60F8E4F5F00422511D40F780ED511D40F170E780ED15
:2001FB00511D40E170E780DD511D50E180D7C39BC5F09C20E70720D207C345F02220D2F9F0
:20021B00D322C5F0C39C7003E5F09B22900E5AE0A360EEE0FFA3E0A3CF2582F582EF358353
:20023B00F58380EBE475F080C0E0C0F01249AC158115815404C5F05400C5F045F0700302B4
:20025B000263E50E547BF50EE475F080C0E0C0F01249AC158115815408C5F05400C5F045AE
:20027B00F07003020287E50E54F7F50E22D28AD2BAD2AAD2AF22C2AA22C0D0C0E0C0F0C0DD
:20029B0083C082C000C001C002C003C004C005C006C0077E3200DEFDA2B35003020327A261
:2002BB00C0400F430F01431410431510908000E514F0A2C150307EFA00DEFDA2C150277E6B
:2002DB00FA00DEFDA2C1501E7EFA00DEFDA2C150157EFA00DEFDA2C1500C7EFA00DEFDA23B
:2002FB00C15003430F02A2C2400F430F04431420431520908000E514F0A2C3400F430F087C
:20031B00431480431580908000E514F0E50F550EF50FD007D006D005D004D003D002D001F3
:12033B00D000D082D083D0F0D0E0D0D0C28BD2AF322209
:05001300C2AF020294DF
:20034E00225388CC5389F0438901758A66758CFCE4F5F0F51685F017E4F5F0F51885F01907
:20036E00E4F5F0F51A85F01BE4F5F0F51C85F01D22D2A9D2B9D2AF43881022C2A95388EFC0
:20038E0022C2AFE4F5F0F51685F017E4F5F0F51A85F01BD2AF22C2AFE4F5F0F51885F0197C
:2003AE00E4F5F0F51C85F01DD2AF2205810581E5168517F078F91200B626C5F00836C5F086
:2003CE00080808F608A6F0124987E5168517F078FD1200B686030886041201ED600302033A
:2003EE00D578FD1200B6E60886F01581158122C2AFC0D0C0E0C0F0C083C082C000C001C014
:20040E0002C003C004C005C006C0075388EF758A66758CFC438810E5168517F0120199F5C4
:20042E001685F0171201A7E5188519F0120199F51885F0191201A7E5188519F07B647C00E0
:20044E0012014045F0600302049BE51E6003020498E50E20E703020495E50F4480F50FE5C5
:20046E00144440F514E5154440F515E475F080C0E0C0F0E51475F000C0E0C0F01249CD1541
:20048E008115811581158102049B751E00E5188519F07BF47C011201DC7003020566E50AA2
:2004AE00050AE50A75F0007B027C00120140F50A7003020506E475F080C0E0C0F0E5157578
:2004CE00F000C0E0C0F01249CD1581158115811581E475F0C0C0E0C0F0E51375F000C0E0F8
:2004EE00C0F01249CD1581158115811581E4F5F0F51885F019020566E475F0C0C0E0C0F094
:20050E00E51275F000C0E0C0F01249CD1581158115811581E475F080C0E0C0F0E51475F02A
:20052E0000C0E0C0F01249CD1581158115811581E4F5F0F51885F019E51A851BF01201993E
:20054E00F51A85F01B1201A7E51C851DF0120199F51C85F01D1201A743871075FF01B2C6D1
:20056E0085900885C009D007D006D005D004D003D002D001D000D082D083D0F0D0E0D0D0B1
:04058E00D2AF322294
:03000B000203FDF0
:1805930022051EC289D2AF3222751E10D288D2B8D2A8D2AF22C2A822BB
:05000300C2AF020594EC
:2005AC0022D2EBD2AFE4900E44F0E4900E43F022C2EB22C0D0C0E0C0F0C083C082C000C08E
:2005CC0001C002C003C004C005C006C0077E3200DEFDA2934003020A65C28CC28DC2A843B5
:2005EC00871075FF01B2C67F0074065388CC5389F0438901758A01758C80D28CCFA293103F
:20060C008D2050F97EFF00DEFDA2C413C2C5A293108D0F40F9D2C5CF1470E1CFC3131304DF
:20062C008005D2C5020A65C28CC28D900E44F043871075FF01B2C67F0074065388CC53896F
:20064C00F0438901758A01758C80D28CCFA293108D1F50F97EFF00DEFDA2C413C2C5A2935C
:20066C00108D0E40F9D2C5CF1470E1CF0303048005D2C5020A65C28CC28D900E43F0438721
:20068C001075FF01B2C6900E47E075F0007B007C001201E47003020767900E46E075F0002D
:2006AC00900E441200D87C001201DC6012900E45E075F000900E431200D87C001201DC45E2
:2006CC00F07003020740900E44E075F000C333C5F033C5F0792A7A001200EA89828A83E097
:2006EC00A3F5F0E0C5F0900E48F0A3C5F0F0C5F0900E43E079007A0075F0001200EA8982DE
:20070C008A83E0900E4AF0900E43E075F000C333C5F033C5F0797C7A001200EA89828A83CC
:20072C00E0A3F5F0E0C5F0900E4DF0A3C5F0F0C5F0020764743475F04E900E48F0A3C5F0E2
:20074C00F0C5F074FF900E4AF0748875F013900E4DF0A3C5F0F0C5F00207D2900E44E0753F
:20076C00F000C333C5F033C5F0792A7A001200EA89828A83E0A3F5F0E0C5F0900E48F0A343
:20078C00C5F0F0C5F0900E43E079007A0075F0001200EA89828A83E0900E4AF0900E43E04D
:2007AC0075F000C333C5F033C5F0797C7A001200EA89828A83E0A3F5F0E0C5F0900E4DF0DA
:2007CC00A3C5F0F0C5F0900E44E0900E46F0900E43E0900E45F0900E47E004900E47F01434
:2007EC0075C500D297C29675C50043C508E5C5541060FA85C61075C500C297C29675C500C0
:20080C0043C508E5C5541060FA85C611900E43E075F0007B407C001201DC700302083D9062
:20082C000E44E075F000C0E0C0F012275115811581900E44E075F0007B217C001201DC7071
:20084C0003020889900E4AE0251175F000900E4BF0A3C5F0F0C5F07BFF7C001201ED700354
:20086C00020880900E4BE0A3F5F0E0C5F0900E4AF002088674FF900E4AF00208BF900E4A98
:20088C00E0251075F000900E4BF0A3C5F0F0C5F07BFF7C001201ED70030208B9900E4BE007
:2008AC00A3F5F0E0C5F0900E4AF00208BF74FF900E4AF0E475F080C0E0C0F01249AC15816D
:2008CC0015815440C5F05400C5F045F0700302090E900E44E075F000C333C5F033C5F07930
:2008EC002A7A001200EA89828A83E0A3F5F0E0C5F07B017C00120187900E48F0A3C5F0F087
:20090C00C5F0E475F080C0E0C0F01249AC158115815420C5F05400C5F045F070030209776E
:20092C00900E44E075F000C333C5F033C5F0792A7A001200EA89828A83E0A3F5F0E0C5F0C3
:20094C00900E48F0A3C5F0F0C5F0900E43E079007A0075F0001200EA89828A83E075F00046
:20096C007B017C00120187900E4AF0E475F080C0E0C0F01249AC158115815420C5F0540038
:20098C00C0F0C0E0E475F080C0E0C0F01249AC158115815440C5F05400C5F01201B3D004C3
:2009AC00D0035BC5F05CC5F045F070030209C8E4F5F0900E4DF0A3C5F0F0C5F0900E4AE053
:2009CC00F5FCD297D296D2A9D28C741B75F000C0E0C0F01249ED15811581742475F001C0FA
:2009EC00E0C0F0124A0D15811581741B75F000C0E0C0F01249ED15811581742B75F001C049
:200A0C00E0C0F0124A0D15811581742E75F001C0E0C0F0900E44E075F000C0E0C0F0900E38
:200A2C0043E075F000C0E0C0F0900E48E0A3F5F0E0C0F0C0E0900E4AE075F000C0E0C0F0D7
:200A4C00900E4DE0A3F5F0E0C0F0C0E0740675F0001248817FF41200C2751E10D288D2A88F
:200A6C00D007D006D005D004D003D002D001D000D082D083D0F0D0E0D0D0C2CBD2EBD2AF4E
:020A8C00322214
:05004B00C2AF0205BF79
:200A8F0022D2E8D2AF22C2E822D2ECD2AF22C2EC22D2EDD2AF22C2ED22C2C8C2E8D2AF32B1
:200AAF00C0D0C0E0743200D5E0FCA2905015430F10431404431504908000E514F0E50F55AE
:200ACF000EF50FD0E0D0D0C2C8C2E8D2AF3222C0D0C0E0431401431501908000E514F0437F
:200AEF000F20E50F550EF50FD0E0D0D0C2CCC2ECD2AF3222C0D0C0E0431402431502908009
:190B0F0000E514F0430F40E50F550EF50FD0E0D0D0C2CDC2EDD2AF322294
:05003300C2AF020AA8A3
:010B290022A9
:05005B00C2AF020ADE45
:010B2B0022A7
:05006300C2AF020B0317
:200B2D0022D2E9D2AF22C2E922C0D0C0E0C0F0C083C082C000C001C002C003C004C005C0A7
:200B4D0006C0077E3200DEFDA2914003020C0FD2AFD297D29675E800D2E8D2ECC2C700D21B
:200B6D00C7900E48E0F5A9A3E0F5C975EA2F43120443130490C000E512F0A291500F438728
:200B8D001075FF01B2C6E50F60F0020C0F743200D5E0FCA29140E3C2EC75F070E50E55F082
:200BAD00B5F05FC2E8C296743200D5E0FC75C50043C50875EA2CC2C700D2C7C2CDD2ED90F6
:200BCD000E4DE0F5AAA3E0F5CA75EA2FE5C5541060FAE5C6C3FEC3740A9E4003020C0FE566
:200BED000F6003020C0F43871075FF01B2C675C50043C508E5C5541060FAE5C6C39E400292
:200C0D0080DDC2ECC2ED75EA2CC2C700D2C75312FB5313FB90C000E512F0C2AFE4F5F0F539
:200C2D001C85F01DE4900E47F0D007D006D005D004D003D002D001D000D082D083D0F0D06F
:0D0C4D00E0D0D075C80075E80ED2AF32229D
:05003B00C2AF020B360C
:200C5B0022D2EAD2AF22C2EA22C0D0C0E0C0F0C083C082C000C001C002C003C004C005C076
:200C7B0006C007743200D5E0FCA2924003020D29D2AFC297D29675E800D2E843120443137E
:200C9B000490C000E512F0A292500F43871075FF01B2C6E50F60F0020D29743200D5E0FCD1
:200CBB00A29240E375F070E50E55F0B5F060C2E8C296745000D5E0FC75C50043C50875EA90
:200CDB002CC2C700D2C7C2CDD2ED900E4DE0F5AAA3E0F5CA75EA2FE5C5541060FAE5C6C34D
:200CFB0013FEC3741E9E4003020D29E50F6003020D2943871075FF01B2C675C50043C508BA
:200D1B00E5C5541060FAE5C6C39E400280DDC2ECC2ED75EA2CC2C700D2C75312FB5313FBDA
:200D3B0090C000E512F0C2AFE4F5F0F51C85F01DE4900E47F0D007D006D005D004D003D0D2
:190D5B0002D001D000D082D083D0F0D0E0D0D075C80075E80ED2AF3222AA
:05004300C2AF020C64D5
:200D75002275E80075EA2C75EB5575EF0075EE0075C80075F83122E475F080C0E0C0F012B0
:200D950049AC158115815401C5F05400C5F045F07003020DB0E50E549FF50EE475F080C031
:200DB500E0C0F01249AC158115815402C5F05400C5F045F07003020DD4E50E54EFF50E2261
:200DD50075E80E2275E800220581058105810581E478FC1200B6F6E4F5F008F608A6F0E47B
:200DF500F514E4F5157402F50EE475F080C0E0C0F01249AC158115815401C5F05400C5F00F
:200E150045F07003020E26E5154401F5154402F515E50E549FF50EE475F080C0E0C0F01232
:200E350049AC158115815402C5F05400C5F045F07003020E54E5154404F5154408F515E4D6
:200E550075F080C0E0C0F01249AC158115815404C5F05400C5F045F07003020E7CE515448D
:200E750020F5154440F515E475F080C0E0C0F01249AC158115815408C5F05400C5F045F00A
:200E95007003020EA0E5154480F515120D761205ADE4F50FC2B5E5124408F512E51344080C
:200EB500F51312038F1203A4E5168517F07BB87C0B1201ED7003020F3DE50920E103020FB3
:200ED50004740A75F000C0E0C0F01203B915811581E50920E103020F0478FC1200B6E6069D
:200EF500E51254F7F512E51354F7F513020F3DE50930E003020F3A740A75F000C0E0C0F07C
:200F15001203B915811581E50930E003020F3A78FC1200B6E606E5144410F514E5154410AA
:200F3500F515020F3D020EBD120DD574FFF50EE4F50F12023F12028812059C120D8C740163
:200F550078FB1200B6F608E66003021104900E4FE075F0007B017C001201E47003021049F4
:200F7500E475F080C0E0C0F01249AC158115815404C5F05400C5F045F06003020FC9E5099A
:200F950030E203020FAB740A75F000C0E0C0F01203B915811581E50930E203020FC978FCED
:200FB5001200B6E606E5144420F514E5154420F515021049E50920E103020FFF740A75F05A
:200FD50000C0E0C0F01203B915811581E50920E103020FFF78FC1200B6E606E51254F7F551
:200FF50012E51354F7F513021049E50930E003021035740A75F000C0E0C0F01203B9158145
:201015001581E50930E00302103578FC1200B6E606E5144410F514E5154410F515021049AC
:20103500E50F700302104678FC1200B6E606021049020F62D29578FC1200B6E660030210E8
:201055006B900E4FE075F0007B017C001201DC700302106BC2B4E50F7003021081E512544C
:20107500F7F512E51354F7F513021104E51C851DF078FD1200B686030886041201FB70038F
:20109500021101E51C851DF018F608A6F0E4F5F079507A0E1200EAC001C002124A34D0836C
:2010B500D082F07B007C001201E470030210C712114FE475F080C0E0C0F01249AC15811562
:2010D500815480C5F05400C5F045F06003021101E51C851DF07B107C0E1201FB7003021100
:2010F50001740A78FC1200B6F602110402106B1205BC120291120DD91205A87402F50EE509
:201115001254F7F512E51354F7F513D2B4C2C574D075F007C0E0C0F01203B915811581D232
:20113500B5D2C515811581158115812275FE0275FCFF75FD8022850BFC220581058105819B
:2011550005810581E4F5F078FA1200B6F608A6F01225901248A15480C5F05400C5F045F04E
:201175007004E5095402700302119478FA1200B6E60886F012019918F608A6F01201A7E4F4
:20119500F5F079507A0E1200EAC001C002124A34D083D082F07B007C001201E470030223DA
:2011B50070E4F5F079507A0E1200EA89828A83E01200FAC0E0C0F0124A48158115819023BD
:2011D50048020103741B75F000C0E0C0F01249ED15811581745775F001C0E0C0F0124A0D0A
:2011F50015811581741B75F000C0E0C0F01249ED15811581745E75F001C0E0C0F0124A0D05
:2012150015811581746175F001C0E0C0F0124A0D15811581E4F50B124A347B207C001201CF
:20123500E4700302136EE50B2404F50B12114B741B75F000C0E0C0F01249ED15811581740D
:20125500A675F001C0E0C0F0124A0D1581158174AE75F001C0E0C0F0E50B75F000C0E0C0FB
:20127500F07402124881158115811581158175C50075C50143C508E5C5541060FA85C60C7C
:2012950075C500741B75F000C0E0C0F01249ED1581158174B275F001C0E0C0F0124A0D15ED
:2012B50081158174BA75F001C0E0C0F0E50C75F000C0E0C0F0740212488115811581158165
:2012D5001581D297C29675C50043C508E5C5541060FA85C60D741B75F000C0E0C0F01249F9
:2012F500ED1581158174BE75F001C0E0C0F0124A0D1581158174C675F001C0E0C0F0E50D61
:2013150075F000C0E0C0F074021248811581158115811581741B75F000C0E0C0F01249EDCE
:201335001581158174CA75F001C0E0C0F0124A0D1581158174D175F001C0E0C0F0E51C8562
:201355001DF0C0E0C0F0740275F000124881158115811581158102122C741B75F000C0E039
:20137500C0F01249ED1581158174D575F001C0E0C0F0124A0D15811581741B75F000C0E00C
:20139500C0F01249ED1581158174DC75F001C0E0C0F0124A0D1581158174DF75F001C0E020
:2013B500C0F0124A0D15811581022370741B75F000C0E0C0F01249ED1581158174E375F0CA
:2013D50001C0E0C0F0124A0D15811581741B75F000C0E0C0F01249ED1581158174EA75F097
:2013F50001C0E0C0F0124A0D1581158174ED75F001C0E0C0F0124A0D15811581747FF50B53
:2014150012114BD297D296124A347B207C001201E47003021509E50820E003021496741B1C
:2014350075F000C0E0C0F01249ED15811581743075F002C0E0C0F0124A0D158115817438D2
:2014550075F002C0E0C0F0124A0D15811581741B75F000C0E0C0F01249ED15811581744DB2
:2014750075F002C0E0C0F0124A0D15811581742A75F000C0E0C0F01249ED1581158102142E
:20149500F6741B75F000C0E0C0F01249ED15811581745575F002C0E0C0F0124A0D158115F5
:2014B50081745D75F002C0E0C0F0124A0D15811581741B75F000C0E0C0F01249ED15811542
:2014D50081747275F002C0E0C0F0124A0D15811581742075F000C0E0C0F01249ED15811508
:2014F5008174C875F000C0E0C0F01203B91581158102141C741B75F000C0E0C0F01249EDAD
:2015150015811581747A75F002C0E0C0F0124A0D15811581741B75F000C0E0C0F01249EDC4
:2015350015811581748175F002C0E0C0F0124A0D15811581748475F002C0E0C0F0124A0D11
:2015550015811581022370741B75F000C0E0C0F01249ED15811581748875F002C0E0C0F04A
:20157500124A0D15811581741B75F000C0E0C0F01249ED15811581748F75F002C0E0C0F04F
:20159500124A0D15811581749275F002C0E0C0F0124A0D15811581D297C296124A347B2063
:2015B5007C001201E4700302160A75C50043C508741B75F000C0E0C0F01249ED158115810C
:2015D50074CC75F002C0E0C0F0124A0D1581158174D475F002C0E0C0F0E50D75F000C0E074
:2015F500C0F07402124881158115811581158185C60D0215B0741B75F000C0E0C0F01249BF
:20161500ED1581158174D875F002C0E0C0F0124A0D15811581741B75F000C0E0C0F0124965
:20163500ED1581158174DF75F002C0E0C0F0124A0D1581158174E275F002C0E0C0F0124A74
:201655000D15811581022370741B75F000C0E0C0F01249ED1581158174E675F002C0E0C0CE
:20167500F0124A0D15811581741B75F000C0E0C0F01249ED1581158174ED75F002C0E0C0F0
:20169500F0124A0D1581158174F075F002C0E0C0F0124A0D15811581747FF50B12114BC2DD
:2016B50097D296124A347B207C001201E470030217A5E50820E003021732741B75F000C058
:2016D500E0C0F01249ED15811581743375F003C0E0C0F0124A0D15811581743B75F003C026
:2016F500E0C0F0124A0D15811581741B75F000C0E0C0F01249ED15811581745175F003C00B
:20171500E0C0F0124A0D15811581742A75F000C0E0C0F01249ED15811581021792741B7519
:20173500F000C0E0C0F01249ED15811581745975F003C0E0C0F0124A0D158115817461757C
:20175500F003C0E0C0F0124A0D15811581741B75F000C0E0C0F01249ED1581158174777584
:20177500F003C0E0C0F0124A0D15811581742075F000C0E0C0F01249ED1581158174C8750E
:20179500F000C0E0C0F01203B9158115810216B8741B75F000C0E0C0F01249ED1581158172
:2017B500747F75F003C0E0C0F0124A0D15811581741B75F000C0E0C0F01249ED158115811C
:2017D500748675F003C0E0C0F0124A0D15811581748975F003C0E0C0F0124A0D1581158163
:2017F500022370741B75F000C0E0C0F01249ED15811581748D75F003C0E0C0F0124A0D1550
:20181500811581741B75F000C0E0C0F01249ED15811581749475F003C0E0C0F0124A0D15A6
:20183500811581749775F003C0E0C0F0124A0D15811581C297C296124A347B207C001201B9
:20185500E470030218A675C50043C508741B75F000C0E0C0F01249ED1581158174D275F0AF
:2018750003C0E0C0F0124A0D1581158174DA75F003C0E0C0F0E50D75F000C0E0C0F0740248
:20189500124881158115811581158185C60D02184C741B75F000C0E0C0F01249ED1581150B
:2018B5008174DE75F003C0E0C0F0124A0D15811581741B75F000C0E0C0F01249ED158115BC
:2018D5008174E575F003C0E0C0F0124A0D1581158174E875F003C0E0C0F0124A0D158115A4
:2018F50081022370741B75F000C0E0C0F01249ED1581158174EC75F003C0E0C0F0124A0D84
:2019150015811581741B75F000C0E0C0F01249ED1581158174F375F003C0E0C0F0124A0D46
:201935001581158174F675F003C0E0C0F0124A0D15811581C297D296E4F50BC2B574FFF52B
:201955001274FFF514124A347B207C001201E47003021FC0E50B2410F50B12114B741B755C
:20197500F000C0E0C0F01249ED15811581742975F004C0E0C0F0124A0D1581158174317599
:20199500F004C0E0C0F0E509540275F0007B017C00120187C0E0C0F0740275F000124881AD
:2019B5001581158115811581741B75F000C0E0C0F01249ED15811581743575F004C0E0C090
:2019D500F0124A0D15811581743D75F004C0E0C0F0E509540475F0007B027C00120187C005
:2019F500E0C0F0740275F0001248811581158115811581741B75F000C0E0C0F01249ED1593
:201A1500811581744175F004C0E0C0F0124A0D15811581744975F004C0E0C0F0E5095408D7
:201A350075F0007B037C00120187C0E0C0F0740275F0001248811581158115811581741BAB
:201A550075F000C0E0C0F01249ED15811581744D75F004C0E0C0F0124A0D15811581745570
:201A750075F004C0E0C0F0E509541075F0007B047C00120187C0E0C0F0740275F0001248C7
:201A9500811581158115811581741B75F000C0E0C0F01249ED15811581745975F004C0E0CA
:201AB500C0F0124A0D15811581746175F004C0E0C0F0E509540175F000C0E0C0F07402755B
:201AD500F0001248811581158115811581741B75F000C0E0C0F01249ED15811581746575C8
:201AF500F004C0E0C0F0124A0D15811581746D75F004C0E0C0F0E508540175F000C0E0C057
:201B1500F0740275F0001248811581158115811581741B75F000C0E0C0F01249ED1581157B
:201B350081747175F004C0E0C0F0124A0D15811581747975F004C0E0C0F0E508540275F08E
:201B5500007B017C00120187C0E0C0F0740275F0001248811581158115811581741B75F08C
:201B750000C0E0C0F01249ED15811581747D75F004C0E0C0F0124A0D15811581748575F0EF
:201B950004C0E0C0F0E508540475F0007B027C00120187C0E0C0F0740275F0001248811584
:201BB50081158115811581741B75F000C0E0C0F01249ED15811581748975F004C0E0C0F05F
:201BD500124A0D15811581749175F004C0E0C0F0E508540875F0007B037C00120187C0E0BB
:201BF500C0F0740275F0001248811581158115811581E508540875F0007B037C00120187D0
:201C150045F07003021C21C2C5021C23D2C5741B75F000C0E0C0F01249ED158115817495A8
:201C350075F004C0E0C0F0124A0D15811581749D75F004C0E0C0F012489B54041200FA7BA3
:201C5500021200F1120187C0E0C0F0740275F0001248811581158115811581741B75F0007E
:201C7500C0E0C0F01249ED1581158174A175F004C0E0C0F0124A0D1581158174A975F004A2
:201C9500C0E0C0F0E50F75F000C0E0C0F074021248811581158115811581741B75F000C0D9
:201CB500E0C0F01249ED1581158174AD75F004C0E0C0F0124A0D1581158174B575F004C04A
:201CD500E0C0F0E50E75F000C0E0C0F074021248811581158115811581741B75F000C0E07A
:201CF500C0F01249ED1581158174B975F004C0E0C0F0124A0D1581158174C175F004C0E0F2
:201D1500C0F0E475F080C0E0C0F01249AC158115815401C5F05400C0F0C0E0740275F00029
:201D35001248811581158115811581741B75F000C0E0C0F01249ED1581158174C575F00401
:201D5500C0E0C0F0124A0D1581158174CD75F004C0E0C0F0E475F080C0E0C0F01249AC155A
:201D75008115815402C5F05400C5F07B017C00120187C0E0C0F0740275F0001248811581F5
:201D9500158115811581741B75F000C0E0C0F01249ED1581158174D175F004C0E0C0F012A4
:201DB5004A0D1581158174D975F004C0E0C0F0E475F080C0E0C0F01249AC158115815404E1
:201DD500C5F05400C5F07B027C00120187C0E0C0F0740275F00012488115811581158115C0
:201DF50081741B75F000C0E0C0F01249ED1581158174DD75F004C0E0C0F0124A0D15811577
:201E15008174E575F004C0E0C0F0E475F080C0E0C0F01249AC158115815408C5F05400C5A4
:201E3500F07B037C00120187C0E0C0F0740275F0001248811581158115811581741B75F0B7
:201E550000C0E0C0F01249ED1581158174E975F004C0E0C0F0124A0D1581158174F175F034
:201E750004C0E0C0F0E475F080C0E0C0F01249AC158115815410C5F05400C5F07B047C0090
:201E9500120187C0E0C0F0740275F0001248811581158115811581741B75F000C0E0C0F0F1
:201EB5001249ED1581158174F575F004C0E0C0F0124A0D1581158174FD75F004C0E0C0F0B8
:201ED500E475F080C0E0C0F01249AC158115815420C5F05400C5F07B057C00120187C0E039
:201EF500C0F0740275F0001248811581158115811581741B75F000C0E0C0F01249ED1581ED
:201F15001581740175F005C0E0C0F0124A0D15811581740975F005C0E0C0F0E475F080C092
:201F3500E0C0F01249AC158115815440C5F05400C5F07B067C00120187C0E0C0F0740275A5
:201F5500F0001248811581158115811581741B75F000C0E0C0F01249ED15811581740D759B
:201F7500F005C0E0C0F0124A0D15811581741575F005C0E0C0F0E475F080C0E0C0F01249BB
:201F9500AC158115815480C5F05400C5F07B077C00120187C0E0C0F0740275F00012488124
:201FB500158115811581158102195AD2B5E4F512E4F514741B75F000C0E0C0F01249ED153F
:201FD500811581741975F005C0E0C0F0124A0D15811581741B75F000C0E0C0F01249ED1558
:201FF500811581742075F005C0E0C0F0124A0D15811581742375F005C0E0C0F0124A0D1503
:20201500811581022370741B75F000C0E0C0F01249ED15811581742775F005C0E0C0F012E0
:202035004A0D15811581741B75F000C0E0C0F01249ED15811581742E75F005C0E0C0F012E2
:202055004A0D15811581743175F005C0E0C0F0124A0D1581158174E875F003C0E0C0F012CE
:2020750003B915811581741B75F000C0E0C0F01249ED15811581747475F005C0E0C0F012F7
:202095004A0D15811581741B75F000C0E0C0F01249ED15811581747B75F005C0E0C0F01235
:2020B5004A0D15811581747E75F005C0E0C0F0124A0D15811581022370741B75F000C0E01E
:2020D500C0F01249ED15811581748275F005C0E0C0F0124A0D15811581741B75F000C0E0EE
:2020F500C0F01249ED15811581748975F005C0E0C0F0124A0D15811581748C75F005C0E051
:20211500C0F0124A0D15811581745075F00EC0E0C0F0740575F000C0E0C0F0124A7A158144
:20213500158115811581745075F00EC0E0C0F0124ADB15811581900E48F0A3C5F0F0C5F00B
:20215500741B75F000C0E0C0F01249ED1581158174B375F005C0E0C0F0124A0D158115813C
:20217500741B75F000C0E0C0F01249ED1581158174BA75F005C0E0C0F0124A0D1581158115
:2021950074BD75F005C0E0C0F0124A0D15811581745075F00EC0E0C0F0740375F000C0E0A7
:2021B500C0F0124A7A1581158115811581745075F00EC0E0C0F0124ADB15811581900E4A5A
:2021D500F0741B75F000C0E0C0F01249ED1581158174E275F005C0E0C0F0124A0D1581151E
:2021F50081741B75F000C0E0C0F01249ED1581158174E975F005C0E0C0F0124A0D15811566
:202215008174EC75F005C0E0C0F0124A0D15811581745075F00EC0E0C0F0740475F000C055
:20223500E0C0F0124A7A1581158115811581745075F00EC0E0C0F0124ADB15811581900E43
:202255004DF0A3C5F0F0C5F0122590741B75F000C0E0C0F01249ED15811581741275F006BF
:20227500C0E0C0F0124A0D15811581741B75F000C0E0C0F01249ED15811581741975F006B4
:20229500C0E0C0F0124A0D15811581741C75F006C0E0C0F0900E48E0A3F5F0E0C0F0C0E07B
:2022B500900E4AE075F000C0E0C0F0900E4DE0A3F5F0E0C0F0C0E0740475F0001248817FD2
:2022D500F81200C202237078FA1200B6E60886F012019918F608A6F01201A7741B75F000E4
:2022F500C0E0C0F01249ED15811581743575F006C0E0C0F0124A0D15811581741B75F00018
:20231500C0E0C0F01249ED15811581743C75F006C0E0C0F0124A0D15811581743F75F006C6
:20233500C0E0C0F0740175F00012488115811581022370DC225800CE2053001B204900F9AE
:20235500184600F81745005D1644005C154300C1134200D91141000000702378FC1200B63B
:20237500E60886F0AB1CAC1D1201E4700302257BE51C851DF018F608A6F0741B75F000C055
:20239500E0C0F01249ED15811581745675F006C0E0C0F0124A0D15811581745C75F006C00F
:2023B500E0C0F0E50875F000C0E0C0F074021248811581158115811581741B75F000C0E099
:2023D500C0F01249ED15811581746075F006C0E0C0F0124A0D15811581746775F006C0E0BA
:2023F500C0F0E50975F000C0E0C0F074021248811581158115811581741B75F000C0E0C078
:20241500F01249ED15811581746B75F006C0E0C0F0124A0D158115811248A178FE1200B6DB
:20243500F6747275F006C0E0C0F0E675F000C0E0C0F0740212488115811581158115817438
:202455001B75F000C0E0C0F01249ED15811581747675F006C0E0C0F0124A0D158115817475
:202475007E75F006C0E0C0F0E50B75F000C0E0C0F07402124881158115811581158175C586
:202495000075C50143C508E5C5541060FA85C60C75C500741B75F000C0E0C0F01249ED1542
:2024B500811581748275F006C0E0C0F0124A0D15811581748A75F006C0E0C0F0E50C75F09B
:2024D50000C0E0C0F074021248811581158115811581D297C29675C50043C508E5C55410D5
:2024F50060FA85C60D741B75F000C0E0C0F01249ED15811581748E75F006C0E0C0F0124A44
:202515000D15811581749675F006C0E0C0F0E50D75F000C0E0C0F074021248811581158184
:2025350015811581741B75F000C0E0C0F01249ED15811581749A75F006C0E0C0F0124A0D70
:202555001581158174A175F006C0E0C0F0E51C851DF0C0E0C0F0740275F00012488115813B
:2025750015811581158178FA1200B6E60886F045F070030211687FFB0200D1741B75F00082
:20259500C0E0C0F01249ED1581158174A575F006C0E0C0F0124A0D15811581741B75F00005
:2025B500C0E0C0F01249ED1581158174A975F006C0E0C0F0124A0D1581158174AC75F0064A
:2025D500C0E0C0F0124A0D1581158174FC75F006C0E0C0F0124A0D15811581744D75F00714
:2025F500C0E0C0F0124A0D15811581749E75F007C0E0C0F0124A0D1581158174EF75F007AF
:20261500C0E0C0F0124A0D15811581744075F008C0E0C0F0124A0D15811581749175F00848
:20263500C0E0C0F0124A0D1581158174E275F008C0E0C0F0124A0D15811581743375F009E3
:20265500C0E0C0F0124A0D15811581748475F009C0E0C0F0124A0D1581158174D575F0097E
:20267500C0E0C0F0124A0D15811581742675F00AC0E0C0F0124A0D15811581747775F00A18
:20269500C0E0C0F0124A0D1581158174C875F00AC0E0C0F0124A0D15811581741975F00BB3
:2026B500C0E0C0F0124A0D15811581746A75F00BC0E0C0F0124A0D1581158174BB75F00B4E
:2026D500C0E0C0F0124A0D15811581740C75F00CC0E0C0F0124A0D15811581745D75F00CE8
:2026F500C0E0C0F0124A0D1581158174AE75F00CC0E0C0F0124A0D1581158174FF75F00C84
:20271500C0E0C0F0124A0D15811581745075F00DC0E0C0F0124A0D1581158174A175F00D1D
:20273500C0E0C0F0124A0D1581158174F275F00DC0E0C0F0124A0D158115812278FB12003B
:20275500B6E61200FA903FDD020103E4F5F079007A001200EAE489828A83F0740175F0008C
:2027750079007A001200EA741E89828A83F0740275F00079007A001200EA741E89828A8347
:20279500F0740375F00079007A001200EA741E89828A83F0740475F00079007A001200EA03
:2027B500741E89828A83F0740575F00079007A001200EA741E89828A83F0740675F00079AB
:2027D500007A001200EA742489828A83F0740775F00079007A001200EA743089828A83F053
:2027F500740875F00079007A001200EA744889828A83F0740975F00079007A001200EA74EB
:202815001E89828A83F0740A75F00079007A001200EA741E89828A83F0740B75F0007900B4
:202835007A001200EA741E89828A83F0740C75F00079007A001200EA741E89828A83F07491
:202855000D75F00079007A001200EA742489828A83F0740E75F00079007A001200EA7430E8
:2028750089828A83F0740F75F00079007A001200EA744889828A83F0741075F00079007AC4
:20289500001200EA745F89828A83F0741175F00079007A001200EA747789828A83F07412FA
:2028B50075F00079007A001200EA748F89828A83F0741375F00079007A001200EA74A78925
:2028D500828A83F0741475F00079007A001200EA74BF89828A83F0741575F00079007A006C
:2028F5001200EA74EE89828A83F0741675F00079007A001200EA74FD89828A83F074177506
:20291500F00079007A001200EAE489828A83F0741875F00079007A001200EAE489828A83FB
:20293500F0741975F00079007A001200EAE489828A83F0741A75F00079007A001200EAE4FF
:2029550089828A83F0741B75F00079007A001200EAE489828A83F0741C75F00079007A00A3
:202975001200EAE489828A83F0741D75F00079007A001200EAE489828A83F0741E75F00092
:2029950079007A001200EAE489828A83F0741F75F00079007A001200EAE489828A83F07400
:2029B5002075F00079007A001200EAE489828A83F0742175F00079007A001200EA74FA89C2
:2029D500828A83F0742275F00079007A001200EA741E89828A83F0742375F00079007A00F0
:2029F5001200EA74FA89828A83F0742475F00079007A001200EA74FA89828A83F0742575E0
:202A1500F00079007A001200EA74FA89828A83F0742675F00079007A001200EA74FA8982E5
:202A35008A83F0742775F00079007A001200EA74FA89828A83F0742875F00079007A001219
:202A550000EA74FA89828A83F0742975F00079007A001200EA74FA89828A83F0E4F5F07958
:202A75002A7A001200EAE4F5F089828A83F0A3C5F0F0C5F0740275F000792A7A001200EADF
:202A9500740A75F00089828A83F0A3C5F0F0C5F0740475F000792A7A001200EA740A75F060
:202AB5000089828A83F0A3C5F0F0C5F0740675F000792A7A001200EA740A75F00089828A8C
:202AD50083F0A3C5F0F0C5F0740875F000792A7A001200EA740A75F00089828A83F0A3C524
:202AF500F0F0C5F0740A75F000792A7A001200EA740A75F00089828A83F0A3C5F0F0C5F048
:202B1500740C75F000792A7A001200EA740A75F00089828A83F0A3C5F0F0C5F0740E75F0D3
:202B350000792A7A001200EA740E75F00089828A83F0A3C5F0F0C5F0741075F000792A7A75
:202B5500001200EA740E75F00089828A83F0A3C5F0F0C5F0741275F000792A7A001200EA74
:202B7500741075F00089828A83F0A3C5F0F0C5F0741475F000792A7A001200EA741475F05F
:202B95000089828A83F0A3C5F0F0C5F0741675F000792A7A001200EA741875F00089828A8D
:202BB50083F0A3C5F0F0C5F0741875F000792A7A001200EA741E75F00089828A83F0A3C51F
:202BD500F0F0C5F0741A75F000792A7A001200EA742475F00089828A83F0A3C5F0F0C5F03D
:202BF500741C75F000792A7A001200EA743075F00089828A83F0A3C5F0F0C5F0741E75F0AD
:202C150000792A7A001200EA743C75F00089828A83F0A3C5F0F0C5F0742075F000792A7A56
:202C3500001200EA744875F00089828A83F0A3C5F0F0C5F0742275F000792A7A001200EA49
:202C5500746075F00089828A83F0A3C5F0F0C5F0742475F000792A7A001200EA747875F0BA
:202C75000089828A83F0A3C5F0F0C5F0742675F000792A7A001200EA749075F00089828A24
:202C950083F0A3C5F0F0C5F0742875F000792A7A001200EA74B475F00089828A83F0A3C598
:202CB500F0F0C5F0742A75F000792A7A001200EA74DC75F00089828A83F0A3C5F0F0C5F094
:202CD500742C75F000792A7A001200EA740E75F00189828A83F0A3C5F0F0C5F0742E75F0CD
:202CF50000792A7A001200EA744075F00189828A83F0A3C5F0F0C5F0743075F000792A7A61
:202D1500001200EA74A475F00189828A83F0A3C5F0F0C5F0743275F000792A7A001200EAFB
:202D3500740875F00289828A83F0A3C5F0F0C5F0743475F000792A7A001200EA746C75F02B
:202D55000289828A83F0A3C5F0F0C5F0743675F000792A7A001200EA743475F00389828A8A
:202D750083F0A3C5F0F0C5F0743875F000792A7A001200EA74FC75F00389828A83F0A3C55C
:202D9500F0F0C5F0743A75F000792A7A001200EA74C475F00489828A83F0A3C5F0F0C5F0B7
:202DB500743C75F000792A7A001200EA745475F00689828A83F0A3C5F0F0C5F0743E75F081
:202DD50000792A7A001200EA74E475F00789828A83F0A3C5F0F0C5F0744075F000792A7AC6
:202DF500001200EA74D875F00989828A83F0A3C5F0F0C5F0744275F000792A7A001200EACF
:202E150074CC75F00B89828A83F0A3C5F0F0C5F0744475F000792A7A001200EA74B475F025
:202E35000F89828A83F0A3C5F0F0C5F0744675F000792A7A001200EA749C75F01389828A14
:202E550083F0A3C5F0F0C5F0744875F000792A7A001200EA748475F01789828A83F0A3C5CF
:202E7500F0F0C5F0744A75F000792A7A001200EA745475F01F89828A83F0A3C5F0F0C5F01B
:202E9500744C75F000792A7A001200EA742475F02789828A83F0A3C5F0F0C5F0744E75F08F
:202EB50000792A7A001200EA74AC75F03A89828A83F0A3C5F0F0C5F0745075F000792A7ADA
:202ED500001200EA743475F04E89828A83F0A3C5F0F0C5F0E4F5F0797C7A001200EAE4F574
:202EF500F089828A83F0A3C5F0F0C5F0740275F000797C7A001200EA746475F00089828AB0
:202F150083F0A3C5F0F0C5F0740475F000797C7A001200EA743C75F00089828A83F0A3C55F
:202F3500F0F0C5F0740675F000797C7A001200EA742875F00089828A83F0A3C5F0F0C5F097
:202F5500740875F000797C7A001200EA741475F00089828A83F0A3C5F0F0C5F0740A75F03B
:202F750000797C7A001200EA740A75F00089828A83F0A3C5F0F0C5F0740C75F000797C7A95
:202F9500001200EA740875F00089828A83F0A3C5F0F0C5F0740E75F000797C7A001200EAE8
:202FB500740675F00089828A83F0A3C5F0F0C5F0741075F000797C7A001200EA740575F0E6
:202FD5000089828A83F0A3C5F0F0C5F0741275F000797C7A001200EA743C75F00089828AD7
:202FF50083F0A3C5F0F0C5F0741475F000797C7A001200EA742875F00089828A83F0A3C583
:20301500F0F0C5F0741675F000797C7A001200EA741475F00089828A83F0A3C5F0F0C5F0BA
:20303500741875F000797C7A001200EA740A75F00089828A83F0A3C5F0F0C5F0741A75F044
:2030550000797C7A001200EA740875F00089828A83F0A3C5F0F0C5F0741C75F000797C7AA6
:20307500001200EA740675F00089828A83F0A3C5F0F0C5F0741E75F000797C7A001200EAF9
:20309500740575F00089828A83F0A3C5F0F0C5F0742075F000797C7A001200EA740575F0F6
:2030B5000089828A83F0A3C5F0F0C5F0742275F000797C7A001200EA740475F00089828A1E
:2030D50083F0A3C5F0F0C5F0742475F000797C7A001200EA740475F00089828A83F0A3C5B6
:2030F500F0F0C5F0742675F000797C7A001200EA740375F00089828A83F0A3C5F0F0C5F0DB
:20311500742875F000797C7A001200EA740375F00089828A83F0A3C5F0F0C5F0742A75F04A
:2031350000797C7A001200EA740275F00089828A83F0A3C5F0F0C5F0742C75F000797C7ABB
:20315500001200EA740275F00089828A83F0A3C5F0F0C5F0742E75F000797C7A001200EA0C
:20317500E4F5F089828A83F0A3C5F0F0C5F0743075F000797C7A001200EAE4F5F089828A9A
:2031950083F0A3C5F0F0C5F0743275F000797C7A001200EAE4F5F089828A83F0A3C5F0F01B
:2031B500C5F0743475F000797C7A001200EAE4F5F089828A83F0A3C5F0F0C5F0743675F0F0
:2031D50000797C7A001200EAE4F5F089828A83F0A3C5F0F0C5F0743875F000797C7A00120F
:2031F50000EAE4F5F089828A83F0A3C5F0F0C5F0743A75F000797C7A001200EAE4F5F08932
:20321500828A83F0A3C5F0F0C5F0743C75F000797C7A001200EAE4F5F089828A83F0A3C564
:20323500F0F0C5F0743E75F000797C7A001200EAE4F5F089828A83F0A3C5F0F0C5F07440E0
:2032550075F000797C7A001200EAE4F5F089828A83F0A3C5F0F0C5F0744275F000797C7A31
:20327500001200EA74D075F00789828A83F0A3C5F0F0C5F0744475F000797C7A001200EA00
:20329500743C75F00089828A83F0A3C5F0F0C5F0744675F000797C7A001200EA743275F06A
:2032B5000089828A83F0A3C5F0F0C5F0744875F000797C7A001200EA742875F00089828AD2
:2032D50083F0A3C5F0F0C5F0744A75F000797C7A001200EA741E75F00089828A83F0A3C574
:2032F500F0F0C5F0744C75F000797C7A001200EA741975F00089828A83F0A3C5F0F0C5F09D
:20331500744E75F000797C7A001200EA741475F00089828A83F0A3C5F0F0C5F0745075F0EB
:2033350000797C7A001200EA740F75F00089828A83F0A3C5F0F0C5F0745275F000797C7A86
:20335500001200EA740A75F00089828A83F0A3C5F0F0C5F0E51254FDF512E51354FDF513D4
:20337500E51254FEF512E51354FEF513023FF1E4F5F079007A001200EAE489828A83F0744C
:203395000175F00079007A001200EA741289828A83F0740275F00079007A001200EA7412E5
:2033B50089828A83F0740375F00079007A001200EA741289828A83F0740475F00079007AC7
:2033D500001200EA741289828A83F0740575F00079007A001200EA741289828A83F0740679
:2033F50075F00079007A001200EA741289828A83F0740775F00079007A001200EA741289F8
:20341500828A83F0740875F00079007A001200EA741289828A83F0740975F00079007A00E5
:203435001200EA741289828A83F0740A75F00079007A001200EA741389828A83F0740B7598
:20345500F00079007A001200EA741889828A83F0740C75F00079007A001200EA741E898273
:203475008A83F0740D75F00079007A001200EA742689828A83F0740E75F00079007A0012D7
:2034950000EA743089828A83F0740F75F00079007A001200EA743C89828A83F0741075F009
:2034B5000079007A001200EA744C89828A83F0741175F00079007A001200EA741289828A4C
:2034D50083F0741275F00079007A001200EA741289828A83F0741375F00079007A0012000B
:2034F500EA741289828A83F0741475F00079007A001200EA741289828A83F0741575F000E7
:2035150079007A001200EA741389828A83F0741675F00079007A001200EA741889828A8396
:20353500F0741775F00079007A001200EA741E89828A83F0741875F00079007A001200EA2D
:20355500742689828A83F0741975F00079007A001200EA743089828A83F0741A75F00079BB
:20357500007A001200EA743C89828A83F0741B75F00079007A001200EA744C89828A83F05D
:20359500741C75F00079007A001200EA745F89828A83F0741D75F00079007A001200EA74FE
:2035B5007789828A83F0741E75F00079007A001200EA749689828A83F0741F75F00079000E
:2035D5007A001200EA74BF89828A83F0742075F00079007A001200EA74EE89828A83F0745F
:2035F5002175F00079007A001200EA74FA89828A83F0742275F00079007A001200EA74FA73
:2036150089828A83F0742375F00079007A001200EA74FA89828A83F0742475F00079007A3C
:20363500001200EA74FA89828A83F0742575F00079007A001200EA74FA89828A83F0742606
:2036550075F00079007A001200EA74FA89828A83F0742775F00079007A001200EA74FA89A5
:20367500828A83F0742875F00079007A001200EA74FA89828A83F0742975F00079007A005B
:203695001200EA74FA89828A83F0E4F5F0792A7A001200EAE4F5F089828A83F0A3C5F0F0A8
:2036B500C5F0740275F000792A7A001200EA740A75F00089828A83F0A3C5F0F0C5F07404EC
:2036D50075F000792A7A001200EA740A75F00089828A83F0A3C5F0F0C5F0740675F0007917
:2036F5002A7A001200EA740A75F00089828A83F0A3C5F0F0C5F0740875F000792A7A00121D
:2037150000EA740A75F00089828A83F0A3C5F0F0C5F0740A75F000792A7A001200EA740A48
:2037350075F00089828A83F0A3C5F0F0C5F0740C75F000792A7A001200EA740A75F00089A0
:20375500828A83F0A3C5F0F0C5F0740E75F000792A7A001200EA740E75F00089828A83F0E9
:20377500A3C5F0F0C5F0741075F000792A7A001200EA740E75F00089828A83F0A3C5F0F0FE
:20379500C5F0741275F000792A7A001200EA741075F00089828A83F0A3C5F0F0C5F07414E5
:2037B50075F000792A7A001200EA741475F00089828A83F0A3C5F0F0C5F0741675F000791C
:2037D5002A7A001200EA741875F00089828A83F0A3C5F0F0C5F0741875F000792A7A00121E
:2037F50000EA741E75F00089828A83F0A3C5F0F0C5F0741A75F000792A7A001200EA74242A
:2038150075F00089828A83F0A3C5F0F0C5F0741C75F000792A7A001200EA743075F0008989
:20383500828A83F0A3C5F0F0C5F0741E75F000792A7A001200EA743C75F00089828A83F0CA
:20385500A3C5F0F0C5F0742075F000792A7A001200EA744875F00089828A83F0A3C5F0F0D3
:20387500C5F0742275F000792A7A001200EA746075F00089828A83F0A3C5F0F0C5F0742494
:2038950075F000792A7A001200EA747875F00089828A83F0A3C5F0F0C5F0742675F00079C7
:2038B5002A7A001200EA749175F00089828A83F0A3C5F0F0C5F0742875F000792A7A0012B4
:2038D50000EA74B475F00089828A83F0A3C5F0F0C5F0742A75F000792A7A001200EA74DCEB
:2038F50075F00089828A83F0A3C5F0F0C5F0742C75F000792A7A001200EA740E75F00189BA
:20391500828A83F0A3C5F0F0C5F0742E75F000792A7A001200EA745475F00189828A83F0C0
:20393500A3C5F0F0C5F0743075F000792A7A001200EA74A475F00189828A83F0A3C5F0F085
:20395500C5F0743275F000792A7A001200EA740875F00289828A83F0A3C5F0F0C5F07434E9
:2039750075F000792A7A001200EA748A75F00289828A83F0A3C5F0F0C5F0743675F00079C2
:203995002A7A001200EA743475F00389828A83F0A3C5F0F0C5F0743875F000792A7A00121D
:2039B50000EA74FC75F00389828A83F0A3C5F0F0C5F0743A75F000792A7A001200EA74F695
:2039D50075F00489828A83F0A3C5F0F0C5F0743C75F000792A7A001200EA745475F006897A
:2039F500828A83F0A3C5F0F0C5F0743E75F000792A7A001200EA74E475F00789828A83F03A
:203A1500A3C5F0F0C5F0744075F000792A7A001200EA74D875F00989828A83F0A3C5F0F058
:203A3500C5F0744275F000792A7A001200EA749475F00C89828A83F0A3C5F0F0C5F0744452
:203A550075F000792A7A001200EA74B475F00F89828A83F0A3C5F0F0C5F0744675F000799A
:203A75002A7A001200EA749C75F01389828A83F0A3C5F0F0C5F0744875F000792A7A0012B4
:203A950000EA74B075F01889828A83F0A3C5F0F0C5F0744A75F000792A7A001200EA74547D
:203AB50075F01F89828A83F0A3C5F0F0C5F0744C75F000792A7A001200EA742475F027897D
:203AD500828A83F0A3C5F0F0C5F0744E75F000792A7A001200EA74E875F03089828A83F01C
:203AF500A3C5F0F0C5F0745075F000792A7A001200EA749475F03E89828A83F0A3C5F0F077
:203B1500C5F0E4F5F0797C7A001200EAE4F5F089828A83F0A3C5F0F0C5F0740275F0007985
:203B35007C7A001200EA746475F00089828A83F0A3C5F0F0C5F0740475F000797C7A0012DE
:203B550000EA745A75F00089828A83F0A3C5F0F0C5F0740675F000797C7A001200EA745020
:203B750075F00089828A83F0A3C5F0F0C5F0740875F000797C7A001200EA744675F00089D2
:203B9500828A83F0A3C5F0F0C5F0740A75F000797C7A001200EA743C75F00089828A83F029
:203BB500A3C5F0F0C5F0740C75F000797C7A001200EA743275F00089828A83F0A3C5F0F048
:203BD500C5F0740E75F000797C7A001200EA742875F00089828A83F0A3C5F0F0C5F074103F
:203BF50075F000797C7A001200EA741E75F00089828A83F0A3C5F0F0C5F0741275F0007980
:203C15007C7A001200EA741475F00089828A83F0A3C5F0F0C5F0741475F000797C7A00123D
:203C350000EA740F75F00089828A83F0A3C5F0F0C5F0741675F000797C7A001200EA740AC0
:203C550075F00089828A83F0A3C5F0F0C5F0741875F000797C7A001200EA740975F000891E
:203C7500828A83F0A3C5F0F0C5F0741A75F000797C7A001200EA740875F00089828A83F06C
:203C9500A3C5F0F0C5F0741C75F000797C7A001200EA740675F00089828A83F0A3C5F0F083
:203CB500C5F0741E75F000797C7A001200EA740575F00089828A83F0A3C5F0F0C5F0742061
:203CD50075F000797C7A001200EA740575F00089828A83F0A3C5F0F0C5F0742275F00079A8
:203CF5007C7A001200EA743275F00089828A83F0A3C5F0F0C5F0742475F000797C7A00122F
:203D150000EA742875F00089828A83F0A3C5F0F0C5F0742675F000797C7A001200EA741EA2
:203D350075F00089828A83F0A3C5F0F0C5F0742875F000797C7A001200EA741475F0008922
:203D5500828A83F0A3C5F0F0C5F0742A75F000797C7A001200EA740F75F00089828A83F074
:203D7500A3C5F0F0C5F0742C75F000797C7A001200EA740A75F00089828A83F0A3C5F0F08E
:203D9500C5F0742E75F000797C7A001200EA740975F00089828A83F0A3C5F0F0C5F074305C
:203DB50075F000797C7A001200EA740875F00089828A83F0A3C5F0F0C5F0743275F00079B4
:203DD5007C7A001200EA740675F00089828A83F0A3C5F0F0C5F0743475F000797C7A00126A
:203DF50000EA740575F00089828A83F0A3C5F0F0C5F0743675F000797C7A001200EA7405EE
:203E150075F00089828A83F0A3C5F0F0C5F0743875F000797C7A001200EA740475F0008941
:203E3500828A83F0A3C5F0F0C5F0743A75F000797C7A001200EA740475F00089828A83F08E
:203E5500A3C5F0F0C5F0743C75F000797C7A001200EA740375F00089828A83F0A3C5F0F0A4
:203E7500C5F0743E75F000797C7A001200EA740375F00089828A83F0A3C5F0F0C5F0744061
:203E950075F000797C7A001200EA740275F00089828A83F0A3C5F0F0C5F0744275F00079C9
:203EB5007C7A001200EA74D075F00789828A83F0A3C5F0F0C5F0744475F000797C7A0012A8
:203ED50000EA743C75F00089828A83F0A3C5F0F0C5F0744675F000797C7A001200EA743299
:203EF50075F00089828A83F0A3C5F0F0C5F0744875F000797C7A001200EA742875F000892D
:203F1500828A83F0A3C5F0F0C5F0744A75F000797C7A001200EA741E75F00089828A83F083
:203F3500A3C5F0F0C5F0744C75F000797C7A001200EA741975F00089828A83F0A3C5F0F09D
:203F5500C5F0744E75F000797C7A001200EA741475F00089828A83F0A3C5F0F0C5F074504F
:203F750075F000797C7A001200EA740F75F00089828A83F0A3C5F0F0C5F0745275F00079CB
:203F95007C7A001200EA740A75F00089828A83F0A3C5F0F0C5F0E5124402F512E5134402B0
:203FB500F513E51254FEF512E51354FEF513023FF17401900E4FF0023FF1E4900E4FF0E5E6
:203FD500154410F515023FF1CF3F0400C63F030084330200602701000000F13F22058105EF
:203FF50081D2B575C50075EB0075A80075E80075B80075F80075870075890075880075EAA0
:204015000075C800E4F512E4F513E4F514E4F5157402F50EE5134410F51312499274807579
:20403500F025C0E0C0F0124B141581158112034F12037F120D76121141124300E4F512E454
:20405500F513E4F514E4F515746475F000900E48F0A3C5F0F0C5F0747F900E4AF07405759F
:20407500F000900E4DF0A3C5F0F0C5F0E5134410F513E4F5F078FD1200B6F608A6F012481B
:20409500A15480C5F05400C5F045F06012E50954021200FA1201BA45F06004E509540170C8
:2040B50003024131740A75F000C0E0C0F01203B9158115811248A15480C5F05400C5F04575
:2040D500F06012E50954021200FA1201BA45F06004E5095401700302410CE4900E47F0E411
:2040F500900E4FF0120DDD74B875F00BC0E0C0F01203B915811581E4F5F078FD1200B6F6F0
:2041150008A6F0748075F025C0E0C0F0124B141581158112034F12037F120D76E50930E0F6
:204135000302414CE5144410F514E5154410F5154410F515024158E51454EFF514E515549E
:20415500EFF515E51C851DF078FD1200B686030886041201FB70030242F8E51C851DF018FE
:20417500F608A6F0124A347B207C001201DC700302418B12114FE475F080C0E0C0F01249D9
:20419500AC158115815401C5F05400C5F045F070030241B6E5154401F5154402F5150241A2
:2041B500E9E5141200FA1201BA5401C5F0E4C5F045F0700FE5141200FA1201BA5402C5F0FB
:2041D500E4C5F045F070030241E9E51554FEF51554FDF515E475F080C0E0C0F01249AC1577
:2041F5008115815402C5F05400C5F045F07003024214E5154404F5154408F515024247E56D
:20421500141200FA1201BA5404C5F0E4C5F045F0700FE5141200FA1201BA5480C5F0E4C53E
:20423500F045F07003024247E51554FBF51554F7F515E475F080C0E0C0F01249AC158115D3
:20425500815404C5F05400C5F045F07003024272E5154420F5154440F5150242A5E514126A
:2042750000FA1201BA5420C5F0E4C5F045F0700FE5141200FA1201BA5440C5F0E4C5F045F3
:20429500F070030242A5E51554DFF51554BFF515E475F080C0E0C0F01249AC1581158154C9
:2042B50008C5F05400C5F045F070030242CCE5154480F5150242E8E5141200FA1201BA5451
:2042D50080C5F0E4C5F045F070030242E8E515547FF515742E75F000C0E0C0F01249ED159C
:2042F5008115810240931581158122E5144401F514E5154401F515E475F080C0E0C0F0E5E1
:204315001475F000C0E0C0F01249CD1581158115811581746475F000C0E0C0F01203B915CF
:20433500811581E5144402F514E5154402F515E475F080C0E0C0F0E51475F000C0E0C0F0F8
:204355001249CD1581158115811581746475F000C0E0C0F01203B915811581E5144404F50B
:2043750014E5154404F515E475F080C0E0C0F0E51475F000C0E0C0F01249CD158115811598
:20439500811581746475F000C0E0C0F01203B915811581E5144408F514E5154408F515E4E8
:2043B50075F080C0E0C0F0E51475F000C0E0C0F01249CD1581158115811581746475F00048
:2043D500C0E0C0F01203B915811581E5144410F514E5154410F515E475F080C0E0C0F0E5D2
:2043F5001475F000C0E0C0F01249CD1581158115811581746475F000C0E0C0F01203B915EF
:20441500811581E5144420F514E5154420F515E475F080C0E0C0F0E51475F000C0E0C0F0DB
:204435001249CD1581158115811581746475F000C0E0C0F01203B915811581E5144440F5EE
:2044550014E5154440F515E475F080C0E0C0F0E51475F000C0E0C0F01249CD15811581157B
:20447500811581746475F000C0E0C0F01203B915811581E5144480F514E5154480F515E417
:2044950075F080C0E0C0F0E51475F000C0E0C0F01249CD1581158115811581746475F00067
:2044B500C0E0C0F01203B915811581E5124401F512E5134401F513E475F0C0C0E0C0F0E5D7
:2044D5001275F000C0E0C0F01249CD1581158115811581746475F000C0E0C0F01203B91510
:2044F500811581E5124402F512E5134402F513E475F0C0C0E0C0F0E51275F000C0E0C0F001
:204515001249CD1581158115811581746475F000C0E0C0F01203B915811581E5124404F54B
:2045350012E5134404F513E475F0C0C0E0C0F0E51275F000C0E0C0F01249CD15811581159E
:20455500811581746475F000C0E0C0F01203B915811581E5124408F512E5134408F513E42E
:2045750075F0C0C0E0C0F0E51275F000C0E0C0F01249CD1581158115811581746475F00048
:20459500C0E0C0F01203B915811581E5124410F512E5134410F513E475F0C0C0E0C0F0E5D8
:2045B5001275F000C0E0C0F01249CD1581158115811581746475F000C0E0C0F01203B9152F
:2045D500811581E51454FEF514E475F080C0E0C0F0E51475F000C0E0C0F01249CD158115C1
:2045F5008115811581746475F000C0E0C0F01203B915811581E51454FDF514E475F080C096
:20461500E0C0F0E51475F000C0E0C0F01249CD1581158115811581746475F000C0E0C0F03A
:204635001203B915811581E51454FBF514E475F080C0E0C0F0E51475F000C0E0C0F01249F8
:20465500CD1581158115811581746475F000C0E0C0F01203B915811581E51454F7F514E468
:2046750075F080C0E0C0F0E51475F000C0E0C0F01249CD1581158115811581746475F00085
:20469500C0E0C0F01203B915811581E51454EFF514E475F080C0E0C0F0E51475F000C0E05F
:2046B500C0F01249CD1581158115811581746475F000C0E0C0F01203B915811581E51454E1
:2046D500DFF514E475F080C0E0C0F0E51475F000C0E0C0F01249CD15811581158115817422
:2046F5006475F000C0E0C0F01203B915811581E51454BFF514E475F080C0E0C0F0E51475F6
:20471500F000C0E0C0F01249CD1581158115811581746475F000C0E0C0F01203B9158115BE
:2047350081E514547FF514E475F080C0E0C0F0E51475F000C0E0C0F01249CD1581158115DE
:20475500811581746475F000C0E0C0F01203B915811581E51254FEF512E51354FEF513E420
:2047750075F0C0C0E0C0F0E51275F000C0E0C0F01249CD1581158115811581746475F00046
:20479500C0E0C0F01203B915811581E51254FDF512E51354FDF513E475F0C0C0E0C0F0E5DC
:2047B5001275F000C0E0C0F01249CD1581158115811581746475F000C0E0C0F01203B9152D
:2047D500811581E51254FBF512E51354FBF513E475F0C0C0E0C0F0E51275F000C0E0C0F00C
:2047F5001249CD1581158115811581746475F000C0E0C0F01203B915811581E51254F7F566
:2048150012E51354F7F513E475F0C0C0E0C0F0E51275F000C0E0C0F01249CD1581158115B8
:20483500811581746475F000C0E0C0F01203B915811581E51254EFF512E51354EFF513E45D
:2048550075F0C0C0E0C0F0E51275F000C0E0C0F01249CD1581158115811581746475F00065
:20487500C0E0C0F01203B9158115812223F42581F8120227124B37120227024A17E580220E
:20489500E59022E5A022E5B022E5C022E5C422E5C822E5ED22E5EC22E5C522E5C55410608C
:2048B500FAE5C622C2AFC2AE75C5000075C50BE5C5541060FAE5C5541060F4E5C6D2AF22A4
:2048D500C2AF7F0074065388CC5389F0438901758A01758C80438810CFA295108D2040F9C1
:2048F5007E5500DEFDA296B313C2C0A295108D0E50F9D2C0CF1470E0CF0303048009538848
:20491500EFD2C07400D2AF22C2AF7F0074065388CC5389F0438901758A01758C80438810E4
:20493500CFA293108D1F50F97E2800DEFDA2C413C2C5A293108D0E40F9D2C5CF1470E1CF25
:2049550003030480095388EFD2C57400D2AF2278FB1200B68603088604741275F07A120169
:20497500461201B1758920F58DF58B75884975985222C2AF43871075FF01D2AF22C2AF431A
:20499500871075FF01B2C6D2AF22C2AF43871075FF01B2C6D2AF2278FB1200B6868208862F
:2049B50083E075F0002278FB1200B68682088683E0F5F0A3E0C5F02278F91200B68682083C
:2049D500868308E6F02278F91200B6868208868308E608F0A3E6F02278FB1200B6E63099FC
:2049F500FDC299F5992274FFF5F030980A3098FDC298E59975F0002278FB1200B686820801
:204A15008683E0602D124A26A380F778FB1200B6E63099FDC299F599B40A17740D80F2E4F3
:204A350030980C3098FDC298E599B40D02740A75F0002278FB1200B6E6C0E008E6C0E012C7
:204A55004CC013D0F0D0E0500224E02278FB1200B6E6C0E008E6C0E0124CC513D0F0D0E045
:204A750050E924202278FC1200B68604188603188683188682E4FDFE124A38B40802800326
:204A9500B47F27ED4E60F11DBDFF011E7408124A267420124A267408124A268583F0E582B2
:204AB5001201A785F083F58280CE124A26F024F3600EA30DBD00010EED8EF01201C070B891
:204AD500E4F0ED8EF02278FB1200B68682088683E4FBFCFFE0A3B42D030FE0A3C39430B4FE
:204AF5000A005012FA740A75F00012012C2AFBE5F03400FC80E4EB8CF0DF030201B12278F4
:204B1500FB1200B68603088604748075F0701201461201B1758920F58DF58B758849759849
:204B35005222124C7E868208868308E4FEFFE07006124C7EE4F022B42551A3E0B42D054310
:204B55000780A3E0B4300343074024D0B40A00500BCE75F00AA42EFEA3E080EEE0B46413AF
:204B7500E60886F030F7084307201201B1A6F018F68003B4750543070A8021B4780543079A
:204B9500108019B46F104307088011124C7EF0A3124C7EA38095B462624307027A00C0043C
:204BB500C005C006C007AB0753031F7C00E60886F0120146A6F018F6EDD007D006D005D04B
:204BD500042430B43A0040022407C0E00AE645F070CC124C7EA902EF30E505742DF0A30A3E
:204BF500124C87D0E0F0A3D9FA0808EF30E7A1EAC39E509C7420F0A30A80F4B4630DAA0143
:204C1500124C7E124C87E6F0A380DEB47331C082C08386820886837A00E06004A30A80F90D
:204C35008683188682124C7E124C87124C7EE0A3124C7E6004F0A380F2D005D00480AAB44A
:204C5500691B86017A00E76004090A80F9124C7E124C878601E76091F009A380F8F97A013B
:204C7500124C7E124C87E9809ECDC583CDCCC582CC22EE601A8FF020F715C002EAC39E5004
:204C95000C742030F6027430F0A30A80EFD00222D005D006124CEC6009C006C00522D005B3
:204CB500D006124CC570F2C006C00590617A802A90415A802590217E802090007F801BD0CB
:204CD50005D006904146124CEF70CE906166124CEF70C6C006C00590303978FB1200B6E6C3
:204CF500B58300400EB5820975F00008E67004042240F5E42278FB1200B6E690001FB47FAE
:204D1500DF80E5D003D004124CA5C004C00370E390207E80C578FB1200B6E6C3940960C89A
:204D35001460C5C3941660C080C9001E1E1E1E1E2430481E1E1E1E2430485F778FA7BFEE50
:204D5500FD00000000000000000000FAFAFAFAFAFAFAFAFA00001400140014001400140013
:204D7500140014001400180018001E001E00240030003C004800600078009000B400DC00A6
:204D95000E014001A40108026C023403FC03C4045406E407D809CC0BB40F9C138417541F16
:204DB5002427AC3A344E000064003C00280014000A000800060005003C00280014000A00B0
:204DD500080006000500050004000400030003000200020000000000000000000000000094
:204DF500000000000000000088133C00320028001E00190014000F000A00000064005A004B
:204E1500500046003C00320028001E0014000F000A0009000800060005000500320028008B
:204E35001E0014000F000A00090008000600050005000400040003000300020088133C000A
:204E5500320028001E00190014000F000A005B32343B3448005B4B0053533E207470636BAB
:204E75003D25642C206370636B3D25642C20543D25642C20493D25642C20546C3D256420F1
:204E9500005B32343B3448005B4B0053533E20444143205357454550204F4E204252454178
:204EB5004B4552205245464552454E4345205349474E414C202D20707265737320535041D0
:204ED500434542415220746F2073746F70202D005B31313B35364800253364005B31323BCA
:204EF50035364800253364005B31333B35364800253364005B353B31384800253564005B30
:204F150032343B3448005B4B0053533E005B32343B3448005B4B0053533E20524458425231
:204F35004B20544553543A20202020202020202020202020202020202020202020202D204A
:204F5500707265737320535041434542415220746F2073746F70202D20005B32343B3231F9
:204F75004800524144494F20425245414B455220414354495645005B31363B313548005B67
:204F950032343B323148002020202020202020202020202020202020202020005B31363B33
:204FB500313548005B32343B3448005B4B0053533E005B32343B3448005B4B0053533E200A
:204FD500524144494F2043555252454E5420544553543A205B2020205D202D207072657311
:204FF5007320535041434542415220746F2073746F70202D20005B32343B3239480025336B
:2050150064005B32343B3448005B4B0053533E005B32343B3448005B4B0053533E20464C61
:205035005242524B20544553543A20202020202020202020202020202020202020202020D0
:20505500202D20707265737320535041434542415220746F2073746F70202D20005B323429
:205075003B32314800464C554F524F20425245414B455220414354495645005B31363B3138
:205095003548005B32343B3231480020202020202020202020202020202020202020202037
:2050B500005B31363B313548005B32343B3448005B4B0053533E005B32343B3448005B4B10
:2050D5000053533E20464C554F524F2043555252454E5420544553543A205B2020205D20AB
:2050F5002D20707265737320535041434542415220746F2073746F70202D20005B32343B6E
:2051150033304800253364005B32343B3448005B4B0053533E005B32343B3448005B4B00F3
:2051350053533E204449474954414C20494E505554205445535420202D207072657373206E
:20515500535041434542415220746F2073746F70202D005B31313B31324800253162005B0D
:2051750031323B31354800253162005B31333B31324800253162005B31343B3135480025EB
:205195003162005B31353B31324800253162005B31363B31354800253162005B31373B3176
:2051B500324800253162005B31383B31354800253162005B31393B31324800253162005B85
:2051D50032303B31354800253162005B31323B33314800253862005B31313B33314800258A
:2051F5003862005B31363B34314800253162005B31363B33384800253162005B31363B3306
:20521500354800253162005B31363B33324800253162005B31363B32394800253162005B1F
:2052350031363B32364800253162005B31363B32334800253162005B31363B323048002521
:205255003162005B32343B3448005B4B0053533E005B32343B3448005B4B0053533E204D35
:20527500792063726561746F7220446F63742E20456E672E2053746566616E6F2047414E6A
:205295005A455454492C207370656369616C207468616E6B7320746F2050494C59005B32A5
:2052B500343B3448005B4B0053533E005B32343B3448005B4B0053533E20494E5055542092
:2052D50074696D65676C6F62616C2056414C55453A5B312E2E32303030305D20005B3234AA
:2052F5003B3448005B4B0053533E20494E5055542063757272676C6F62616C2056414C5503
:20531500453A5B302E2E3235355D20005B32343B3448005B4B0053533E20494E5055542027
:20533500636F6461676C6F62616C2056414C55453A5B312E2E323030305D20005B32343B56
:205355003448005B4B0053533E20543D2564203B20493D2564203B20546C3D256420005BF2
:2053750032343B3448005B4B0053533E204259452E2E2E2E2E2E2E2E2E2E2E2E2E2E2000CD
:205395005B373B394800253862005B373B34394800253862005B373B363948002538620067
:2053B5005B31313B35364800253364005B31323B35364800253364005B31333B353648005C
:2053D500253364005B353B31384800253564005B324A005B4800CDCDCDCDCDCDCDCDCDCD46
:2053F500CDCDCDCDCDCDCDCDCDCDCDCDCDCDCDCDCDCDCDCDCDCDCDCDCDCDCDCDCDCDCDCDF8
:20541500CDCDCDCDCDCDCDCDCDCDCDCDCDCDCDCDCDCDCDCDCDCDCDCDCDCDCDCDCDCDCDCDD7
:20543500CDCDCDCDCD000AB0B0B0B1B1B2205341464554592053555045525649534F5220DA
:20545500B2B1B1B0B0B020202020202020202020202020666F7220626F61726420526576B7
:205475002E3420202020202020205B53787830312E3030385D20000ACDCDCDCDCDCDCDCD01
:20549500CDCDCDCDCDCDCDCDCDCDCDCDCDCDCDCDCDCDCDCDCDCDCDCDCDCDCDCDCDCDCDCD57
:2054B500CDCDCDCDCDCDCDCDCDCDCDCDCDCDCDCDCDCDCDCDCDCDCDCDCDCDCDCDCDCDCDCD37
:2054D500CDCDCDCDCDCDCD000A202020202020202020202020202020202020202020202032
:2054F500202020202020202020202020202020202020202020202020202020202020202097
:20551500202020202020202020202020202020202020202020202020000A20C420E643201F
:20553500535441545553206174205B20202020205D20C4C4C4C4C4C4C4C4C4C4C4C4C4C42D
:20555500C4C4C4C4C4C4C4C4C4C4C4C4C4C4C4C4C4C4C4C4C4C4C4C4C4C4C4C4C4C4C4C4B6
:20557500C4C4C4C4C4C4C4C4C4000A20202020202020202020202020202020202020202088
:205595002020202020202020202020202020202020202020202020202020202020202020F6
:2055B5002020202020202020202020202020202020202020202020202020000A20202050DC
:2055D50031203A5B20202020202020205D2020202020202050333A5B20202020202020207B
:2055F5005D2020202020202050343A5B20202020202020205D2020202020202050353A5BE9
:2056150020202020202020205D2020000A202020202020202020202020202020202020206E
:20563500202020202020202020202020202020202020202020202020202020202020202055
:2056550020202020202020202020202020202020202020202020202020202020000A20C4C7
:20567500204449474954414C2053454354494F4E20C4C4C4C4C4C4C4C4C4C4C4C4C4C4C426
:20569500C4C4C4C4C4C4C4C4202020C420414E414C4F472053454354494F4E20C4C4C4C47A
:2056B500C4C4C4C4C4C4C4C4C4C4C4C4C4000A2020202020202020202020202020202020B7
:2056D5002020202020202020202020202020202020202020202020202020202020202020B5
:2056F500202020202020202020202020202020202020202020202020202020202020000ACB
:205715002020204F4646202020205B205D202020202020616C726D5F6D736B203A5B2020D6
:205735002020202020205D20202020202020206876636472763A5B2020205D2020202020B8
:20575500202020202020202020202020202020000A202020755341462020202020205B2060
:205775005D202020616C726D5F6D7367203A5B20202020202020205D2020202020202020F3
:2057950068766664626B3A5B2020205D2020202020202020202020202020202020202020AD
:2057B500000A20202046494C534146205B205D20202020202020202020202020202020209D
:2057D50020202020202020202020202020202020206876637572723A5B2020205D20202048
:2057F5002020202020202020202020202020202020000A2020204441544120202020202030
:205815005B205D2020202020202020202020202020202020202020202020202020202020FB
:20583500202020202020202020202020202020202020202020202020202020202020202053
:205855002020000A2020204C494E452020205B205D20202020202020202020202020202049
:205875002020202020202020202020202020202020C4204B45595354524F4B45204D454E4E
:205895005520C4C4C4C4C4C4C4C4C4C4C4C4C4C4C4C4C4000A20202042524B202020202091
:2058B50020205B205D20205B205D5B205D5B205D5B205D5B205D5B205D5B205D5B205D209B
:2058D5002020202020202020202020202020202020202020202020202020202020202020B3
:2058F50020202020000A2020205258544D2020205B205D2020202020204A20204A20204A08
:2059150020204A20204A20204A20204A20204A20202020202027412720444143205357457A
:205935004550202020202027452720464C554F524F20524420000A202020464C544D2020E0
:20595500202020205B205D202020502020502020502020502020502020502020502020503A
:2059750020202020202027422720524144494F2042524B20202020202746272044494749C3
:20599500542054535420000A2020205354524F4245205B205D2020202020202020202020D2
:2059B500203120203120203120203120203120203120202020202027432720524144494F6C
:2059D50020524420202020202027532720534552205041524D5320000A2020205744202089
:2059F5002020202020205B205D20202038202039202030202031202032202033202034208F
:205A1500203520202020202027442720464C554F524F2042524B202020202749276E666F7A
:205A35002020202020202020000A2020202020202020202020202020202020202020202087
:205A5500202020202020202020202020202020202020202020202020202020202020202031
:205A750020202020202020202020206527582769742020202020202020000A20202020201F
:205A95002020202020202020202020202020202020202020202020202020202020202020F1
:205AB5002020202020202020202020202020202020202020202020202020202020202020D1
:205AD50020202020202020202020000A20C4C4204D455353414745204152454120C4C4C4F5
:205AF500C4C4C4C4C4C4C4C4C4C4C4C4C4C4C4C4C4C4C4C4C4C4C4C4C4C4C4C4C4C4C4C411
:205B1500C4C4C4C4C4C4C4C4C4C4C4C4C4C4C4C4C4C4C4C4C4C4C4C4C4C4C4000A2020205A
:205B350053533E2020202020202020202020202020202020202020202020202020202020CC
:205B5500202020202020202020202020202020202020202020202020202020202020202030
:0D5B750020202020202020202020202000A3
:00000001FF
